:1000000000000000000000000C06060000040600CE
:100010000C060602000406000C0606040004060096
:100020000C060606000406000C060608000406007E
:100030000C06060A000406000C06060C0004060066
:100040000C06060E000406000C060600010406005D
:100050000C060602010406000C0606040104060054
:100060000C060606010406000C060608010406003C
:100070000C06060A010406000C06060C0104060024
:100080000C06060E010406000C060600020406001B
:100090000C060602020406000C0606040204060012
:1000A0000C060606020406000C06060802040600FA
:1000B0000C06060A020406000C06060C02040600E2
:1000C0000C06060E020406000C06060003040600D9
:1000D0000C060602030406000C06060403040600D0
:1000E0000C060606030406000C06060803040600B8
:1000F0000C06060A030406000C06060C03040600A0
:100100000C06060E030406000C0606000404060096
:1001100000070602000406000007060400040600AB
:100120000007060600040600000706080004060093
:100130000007060A000406000007060C000406007B
:100140000007060E00040600000706000104060072
:100150000007060201040600000706040104060069
:100160000007060601040600000706080104060051
:100170000007060A010406000007060C0104060039
:100180000007060E01040600000706000204060030
:100190000007060202040600000706040204060027
:1001A000000706060204060000070608020406000F
:1001B0000007060A020406000007060C02040600F7
:1001C0000007060E020406000007060003040600EE
:1001D00000070602030406000007060403040600E5
:1001E00000070606030406000007060803040600CD
:1001F0000007060A030406000007060C03040600B5
:100200000007060E030406000007060004040600AB
:1002100004070602000406000407060400040600A2
:10022000040706060004060004070608000406008A
:100230000407060A000406000407060C0004060072
:100240000407060E00040600040706000104060069
:100250000407060201040600040706040104060060
:100260000407060601040600040706080104060048
:100270000407060A010406000407060C0104060030
:100280000407060E01040600040706000204060027
:10029000040706020204060004070604020406001E
:1002A0000407060602040600040706080204060006
:1002B0000407060A020406000407060C02040600EE
:1002C0000407060E020406000407060003040600E5
:1002D00004070602030406000407060403040600DC
:1002E00004070606030406000407060803040600C4
:1002F0000407060A030406000407060C03040600AC
:100300000407060E030406000407060004040600A2
:100310000807060200040600080706040004060099
:100320000807060600040600080706080004060081
:100330000807060A000406000807060C0004060069
:100340000807060E00040600080706000104060060
:100350000807060201040600080706040104060057
:10036000080706060104060008070608010406003F
:100370000807060A010406000807060C0104060027
:100380000807060E0104060008070600020406001E
:100390000807060202040600080706040204060015
:1003A00008070606020406000807060802040600FD
:1003B0000807060A020406000807060C02040600E5
:1003C0000807060E020406000807060003040600DC
:1003D00008070602030406000807060403040600D3
:1003E00008070606030406000807060803040600BB
:0803F0000807060A03040600D9
:100400000000000000000000010B0C0000000504CB
:10041000010B0C0400000504010B0C020000050494
:10042000010B0C0600000504010B0C010000050483
:10043000010B0C0500000504010B0C030000050472
:10044000010B0C0700000504010B0C00080005045B
:10045000010B0C0408000504010B0C020800050444
:10046000010B0C0608000504010B0C010800050433
:10047000010B0C0508000504010B0C030800050422
:10048000010B0C0708000504010B0C000400050417
:10049000010B0C0404000504010B0C02040005040C
:1004A000010B0C0604000504010B0C0104000504FB
:1004B000010B0C0504000504010B0C0304000504EA
:1004C000010B0C0704000504010B0C000C000504D3
:1004D000010B0C040C000504010B0C020C000504BC
:1004E000010B0C060C000504010B0C010C000504AB
:1004F000010B0C050C000504010B0C030C0005049A
:10050000010B0C070C000504010B0C000200050494
:10051000010B0C0402000504010B0C02020005048F
:10052000010B0C0602000504010B0C01020005047E
:10053000010B0C0502000504010B0C03020005046D
:10054000010B0C0702000504010B0C000A00050456
:10055000030B0C0400000504030B0C02000005044F
:10056000030B0C0600000504030B0C01000005043E
:10057000030B0C0500000504030B0C03000005042D
:10058000030B0C0700000504030B0C000800050416
:10059000030B0C0408000504030B0C0208000504FF
:1005A000030B0C0608000504030B0C0108000504EE
:1005B000030B0C0508000504030B0C0308000504DD
:1005C000030B0C0708000504030B0C0004000504D2
:1005D000030B0C0404000504030B0C0204000504C7
:1005E000030B0C0604000504030B0C0104000504B6
:1005F000030B0C0504000504030B0C0304000504A5
:10060000030B0C0704000504030B0C000C0005048D
:10061000030B0C040C000504030B0C020C00050476
:10062000030B0C060C000504030B0C010C00050465
:10063000030B0C050C000504030B0C030C00050454
:10064000030B0C070C000504030B0C00020005044F
:10065000030B0C0402000504030B0C02020005044A
:10066000030B0C0602000504030B0C010200050439
:10067000030B0C0502000504030B0C030200050428
:10068000030B0C0702000504030B0C000A00050411
:1006900000070C040000050400070C02000005041C
:1006A00000070C060000050400070C01000005040B
:1006B00000070C050000050400070C0300000504FA
:1006C00000070C070000050400070C0008000504E3
:1006D00000070C040800050400070C0208000504CC
:1006E00000070C060800050400070C0108000504BB
:1006F00000070C050800050400070C0308000504AA
:1007000000070C0708000504030B0C000800050493
:10071000030B0C0408000504030B0C02080005047D
:10072000030B0C0608000504030B0C01080005046C
:10073000030B0C0508000504030B0C03080005045B
:10074000030B0C0708000504030B0C000400050450
:10075000030B0C0404000504030B0C020400050445
:10076000030B0C0604000504030B0C010400050434
:10077000030B0C0504000504030B0C030400050423
:10078000030B0C0704000504030B0C000C0005040C
:1007900000070C040200050400070C020200050417
:1007A00000070C060200050400070C010200050406
:1007B00000070C050200050400070C0302000504F5
:1007C00000070C070200050402070C0000000504E6
:1007D00002070C040000050402070C0200000504D7
:1007E00002070C060000050402070C0100000504C6
:1007F00002070C050000050402070C0300000504B5
:0807F80002070C0700000504D4
:00000001FF
